:1000000019C032C031C030C030C02EC02DC02CC08D
:100010002BC02AC029C028C027C0B4C025C024C016
:1000200096C022C021C020C01FC01EC01DC01CC061
:100030001BC01AC011241FBECFEFD4E0DEBFCDBF5E
:1000400011E0A0E0B1E0E6E6F2E002C005900D921A
:10005000A031B107D9F711E0A0E1B1E001C01D92D4
:10006000A131B107E1F79EC0CBCF1F920F920FB61F
:100070000F9211248F939F93EF93FF934C9B02C099
:1000800030993AC080911001833009F455C08091B5
:100090001001882309F450C080911001823009F4C6
:1000A00042C080916400877F8093640081E090E08B
:1000B0009093890080938800E9B1FF27E770F07082
:1000C000EE0FFF1FE050FF4F8081918190938B00D6
:1000D00080938A0080EF80938000109268001092D5
:1000E00085001092840081E080936F0080938100EE
:1000F00083E08093100120C080911001813011F6BF
:1001000082E080931001319BFECF90E895B98091F9
:1001100064008F7D8093640096BD81E080936E00C3
:1001200084E085BD09C015BC10926E00809164000A
:10013000806280936400B5CF82E08BBBFF91EF912A
:100140009F918F910F900FBE0F901F9018951F9247
:100150000F920FB60F9211248F93EF93FF9381E0CC
:100160008093100115BC10926E00E4E6F0E08081EF
:1001700080628083FF91EF918F910F900FBE0F905F
:100180001F9018951F920F920FB60F921124109284
:1001900010011092810010926F000F900FBE0F900F
:1001A0001F901895CFEFD4E0DEBFCDBF10921001A5
:1001B00080EE8AB98FE18BB98CE787B983E088B983
:1001C00080936C008FEF84B915B810928000109264
:1001D000810080E880BF809164008F6E809364000E
:1001E00080916400877F8093640050EA60EC21E096
:1001F00030E092E041E050938000109281006093E3
:10020000820016BC109280003093890020938800F1
:10021000909368009BBB7894809164008860809381
:1002200064004093100180911001882369F419C083
:10023000813028F0843018F483B7817F83BF88959C
:1002400080911001882369F080911001813081F73D
:1002500083B7817F846083BF889580911001882354
:0602600099F7F894C8CFE5
:10026600D007AF0058002C0012000A00050003005A
:00000001FF
